:1000000012C02CC02BC02AC029C028C027C026C0BF
:1000100025C02CC023C022C021C020C01FC01EC0CC
:100020001DC01CC01BC011241FBECFE5D4E0DEBF25
:10003000CDBF10E0A0E6B0E0E4E1F1E002C0059041
:100040000D92A036B107D9F710E0A0E6B0E001C0EC
:100050001D92A436B107E1F74BD05AC0D1CF83B778
:10006000836083BF89B7816089BF08951F920F9213
:100070000FB60F9211248F939F9383E882BF8091D4
:100080006000909161000196909361008093600000
:1000900080916000909161008436910569F410921E
:1000A000610010926000809162009091630001965F
:1000B000909363008093620080916200909163004E
:1000C000449779F4109263001092620082B38058D2
:1000D00082BB82B391E0892782BB82B392E08927F9
:1000E00082BB9F918F910F900FBE0F901F9018951C
:1000F0008F9A889A899A909A919A979A909A9198B9
:1001000083B7836083BF89B7816089BF7894FFCF4D
:04011000F894FFCF91
:00000001FF
